:10000000830100308A00042883010A128A11E52B3B
:10001000C400C51B1428451B1C2845088A00440839
:10002000C40A0319C50A82008313451883174408BC
:10003000C40A840000080800423469346C3469340E
:100040006D342034763465342034543465346B3464
:100050006E3469346B340034253464342E342534E2
:10006000643443342034003482070034A0343B34F9
:10066000031383120800F0000030711870070310A4
:10067000F00D0310F10CF10803190800352BF401FB
:10068000F5010310F30CF20C031C4D2B7008F4075A
:1006900071080318710AF5070310F00DF10D7208C7
:1006A000730403190034412B83120313A0000515B2
:1006B000200E0F39F0000608F03970048600851509
:1006C000851120080F39F0000608F0397004860003
:1006D000851585110D30A100A10B6C2B080083122C
:1006E0000313B800380E0F39F0000608F039700413
:1006F00086008515851138080F39F0000608F03995
:1007000070048600851585110D30B900B90B862B54
:10071000080083120313051101306F230230B22B3E
:10072000831203130515A02B3708C5003608B60A37
:100730000319B70A0A128A1108200A128A116F23B4
:100740003708C50036080A128A1108200A128A11D1
:10075000003803190800942B83120313B600051107
:10076000803E6F2B83120313B7000430B800533060
:10077000B900B90BB92BB80BB72BB70BB52B0800C9
:100780008312031305110F30B22303308600851541
:1007900085110530B223851585112130B600B60BC1
:1007A000CF2B851585110530B223023086008515C3
:1007B00085110D30B600B60BDB2B28306F230830C7
:1007C0006F230F306F2306306F2B533083120313C8
:1007D000A6004930A7004330A8004130A9004B30A3
:1007E000AA004C30AB004930AC004B30AD0020309B
:1007F000AE003D30AF002030B000B101831686015D
:1008000001308500FA30B223C0230A128A118923ED
:100810000A128A118E3083169F00413083129F0086
:1008200045309F001F19122C1E08A2000030F10055
:1008300022080A128A11332383161E078312A2008C
:10084000F0000A128A11BA26F301C830F4004230CF
:10085000F5000A128A110B270030C50035300A1244
:100860008A110820F3000A128A110920F4000A12E2
:100870008A110920F5000A128A110B277008A300BB
:100880007108A4007208A5002308F0002408F100F4
:100890002508F2000A128A114C277008A100F00006
:1008A0000A128A11BA267008F3007108F40072085F
:1008B000F5002308F0002408F1002508F2000A12D0
:1008C0008A11E926F3012030F4004130F5000A12C4
:1008D0008A110B270A128A114C277008A0002C30AD
:1008E000B7000030B8002008B400B5012108B200FC
:1008F000B3013230B60031300A128A1199240A123B
:100900008A110030AC230A128A111C30B600003064
:10091000B70090234030AC230A128A112630B6006B
:100920008030B7009023FA30B22389230A128A114B
:10093000102C83120313BF00BD013608BA008D2EA0
:100940003E08253A031D7E2EFF30BB00BC01B901D5
:10095000402EBF080319B02C3F0884008313800188
:100960003D0808000230BA073A02840083130008E9
:100970007C2EB90ABF2C0830BB07FE30BB07023003
:10098000BA073A02840083130008C000840A0008F2
:10099000C1003918C11FD32CC009C109C00A0319ED
:1009A000C10ABC03D42CB9010B30BB073B08F200D1
:1009B000F3014108F1004008F0000A128A11BB2738
:1009C0007008BE003B08F200F3014008F000410847
:1009D000F1000A128A11BB270A128A117408C0009A
:1009E0007508C100C201C20AC30143084102031DC8
:1009F000FB2C42084002031C202D3B08F200F301AF
:100A00004208F0004308F1000A128A113F230A123B
:100A10008A117408C2007508C300BC03F52CBD0A16
:100A2000BF0803191A2D3F0884008313203080006B
:100A3000BF0A202D20300A128A1130230A128A118F
:100A4000BC033C08803A7F3E03180F2D391C372D1C
:100A5000BD0ABF080319332D3F08840083132D30CE
:100A60008000BF0A372D2D300A128A1130233B082F
:100A7000F200F3014208F0004308F1000A128A1163
:100A8000BB270A128A117408C2007508C300420409
:100A90000319762D4308F3004208F2004108F100E3
:100AA0004008F0000A128A11BB277408F00075088C
:100AB000F1003B08F200F3010A128A11BB270A1267
:100AC0008A117008BC00803A763E031C692D0730FD
:100AD000BC07BD0ABF080319732D3F0884008313A8
:100AE0003C08303E302D3C08303E342D0A303E026A
:100AF000031C7C2D0730BE07BD0ABF080319862DD5
:100B00003F08840083133E08303E862E3E08303E68
:100B10008A2EBD0ABF080319942D3F088400831351
:100B200020308000BF0A9A2D20300A128A1130230B
:100B30000A128A11BC033C08803A7E3E0318892DB4
:100B40000230BA073A02840083130008BE007E2EEA
:100B50000230BA073A02840083130008C200840AF4
:100B60000008C300BE013E084207C4004308C50098
:100B700044080318C50A0A128A1108200A128A11A9
:100B800000380319C52DBE0AB32D3B083E020318D9
:100B9000CB2D3E08BB003B08BC1B022EFF3A3C0796
:100BA000031C022EBD0ABF080319DD2D3F08840077
:100BB000831320308000BF0AE32D20300A128A11EF
:100BC00030230A128A11BC03CB2D4308C50042080A
:100BD0000A128A1108200A128A11BE00C20A0319D9
:100BE000C30ABD0ABF080319FC2D3F088400831304
:100BF0003E088000BF0A022E3E080A128A113023E6
:100C00000A128A11BB033B0FE52D8D2E3808C50053
:100C100037080A128A1108200A128A112A3A031D7B
:100C2000182E0230BA073A028400831300083C2EC3
:100C30003808C50037080A128A110820D03EBB00C8
:100C4000B70A0319B80A3808C50037080A128A110A
:100C500008200A128A11BE0030303E02031C402ECA
:100C60003A303E020318402E0A30F1003B080A12C7
:100C70008A1133233E07D03EBB00B70A0319B80AD6
:100C80003808C5003708B70A0319B80A0A128A11CA
:100C900008200A128A11BE00003A0319A92C2A3A28
:100CA0000319B22C043A0319062E763A0319BB2C09
:100CB0003B3A03199B2D073A0319B92C0B3A031938
:100CC000BD2C1C3A0319A82D063A0319BF2C0D3A66
:100CD0000319BB2C30303E02031C7E2E3A303E02FC
:100CE00003187E2E0A30F1003C080A128A113323C1
:100CF0000A128A113E07D03EBC00402EBD0ABF0832
:100D00000319892E3F08840083133E088000BF0A20
:100D10008D2E3E080A128A1130233808C500370884
:100D2000B70A0319B80A0A128A1108200A128A118E
:100D3000BE00BE08031DA02CBF080319A32E3F0848
:100D40008400831380013D080800840803190034DF
:100D5000720880008403710880008403700880009A
:100D60000034F101F201F301F01FC32EF103F2038D
:100D7000F303BE2EF101F201F301C32EF31FC32EC4
:100D80007814F227C42EF8018E30F6008401F3089F
:100D90000319992F0310F30CF20CF10CF00CF60A66
:100DA000C72E76087702031CE02E031908000310F3
:100DB000F20CF10CF00CF60A76087702D52E03102F
:100DC000F50CF40CF30CF70A760877060319080003
:100DD000DF2E8030F50684016F277E27D126781814
:100DE000F227F81CFB2EF309F409F509F30A03199D
:100DF000F40A0319F50A7308F00774080318740F4E
:100E0000F10775080318750FF207F801F21F992F03
:100E1000F2277814992F84016F277E27F901FA01B0
:100E2000FB010730F5000310F40CF30C031C232F17
:100E30007008F90771080318710FFA077208031890
:100E4000720FFB070310F00DF10DF20DF50B132FD0
:100E50000930F5002F2F0310FB0CFA0CF90C0310CE
:100E6000F40CF30C031C3E2F7008F90771080318EB
:100E7000710FFA0772080318720FFB07F50B2B2F7F
:100E80007A307707F607780CF8067908F0007A08C8
:100E9000F1007B08F200992F84016F27F301823063
:100EA000F607F61B7A2FF030F607F61B682F18307E
:100EB000760203187A2FF608031D612F7818F2279F
:100EC0000800F6030310F00DF10DF20DF30D5B2F8A
:100ED0000310F20CF10CF00CF60F682F5E2FF801E6
:100EE000710D720DF600003803197A2FF80DF2011A
:100EF000F1170800F001F101F2010034F810740D4F
:100F0000750DF700003803198A2F0318F814F5013E
:100F1000F4170800F701F301F401F5010800760861
:100F200003197A2FF113F80C760CF2000318F1175D
:100F3000A52EF608031DAD2FF001F101F201A52E3B
:100F400072030319F00A0319F10A0319F20A0310D4
:100F5000F20CF10CF00CF60A992FF208031DA02FE9
:100F60007008710403199C2FF11B8F2FF6030310D7
:100F7000F00DF10DB42FF601F401F50172087304C0
:100F8000031900341F30F6040310F60AF20DF30DB6
:100F9000031CC52FF30CF20C73087102031DD22F32
:100FA00072087002031CDA2F7208F0027308031C27
:100FB000730AF102F40DF50DF60BF61ACA2FF61F9F
:100FC000E62FF409F40A0319F503F5097408F20091
:100FD0007508F300761F0034F009F00A0319F103D5
:100FE000F10900340310FF30F007F009031CF1078A
:100FF000F109031CF207F209031CF307F3090800C7
:00000001FF
